:020000040000FA
:10000000831285010730990083169F012C308500EB
:100010008312FF308500043032203C3029204930E3
:100020001D20122800308500FA303220CE303220D8
:100030001230292070301D200928F13EA000201820
:100040002128A0182328A0182528FC3E03182528BD
:100050000800FF3EA1005E301D2060301D20A10B76
:100060002D280800FF3EA200633029205D301D20AE
:10007000633029205F301D20A20B38280800432060
:100080004420442043204420472000000000080072
:02400E00D33F9E
:00000001FF
